:0200000480007A
:100000006F008004732F2034930F80006308FF0378
:10001000930F90006304FF03930FB0006300FF038E
:10002000130F000063040F0067000F00732F2034CC
:1000300063540F006F00400093E19153171F0000BD
:1000400023223FFC6FF09FFF93000000130100008C
:10005000930100001302000093020000130300004C
:100060009303000013040000930400001305000034
:10007000930500001306000093060000130700001C
:100080009307000013080000930800001309000004
:1000900093090000130A0000930A0000130B0000EC
:1000A000930B0000130C0000930C0000130D0000D4
:1000B000930D0000130E0000930E0000130F0000BC
:1000C000930F0000732540F16310050097020000B4
:1000D000938202017390523073500018970200000F
:1000E0009382020273905230B70200809382F2FF33
:1000F0007390023B9302F0017390023A73504030C8
:100100009702000093824201739052307350203066
:100110007350303093010000970200009382C2EECA
:1001200073905230130510001315F501634C050050
:100130000F00F00F930110009308D0051305000085
:100140007300000093020000638A02007390521053
:10015000B7B2000093829210739022307350003037
:10016000970200009382420173901234732540F18C
:1001700073002030972000009380C0E803D7000070
:100180009303F00F93012000631677269720000059
:10019000938040E703D72000B7030100938303F067
:1001A000930130006318772497200000938080E546
:1001B00003D74000B7130000938303FF930140006F
:1001C000631A7722972000009380C0E303D7600072
:1001D000B7F300009383F30093015000631C772072
:1001E00097200000938060E203D7A0FF9303F00FF5
:1001F0009301600063107720972000009380E0E077
:1002000003D7C0FFB7030100938303F0930170008D
:100210006312771E97200000938020DF03D7E0FF52
:10022000B7130000938303FF930180006314771CCE
:1002300097200000938060DD03D70000B7F3000033
:100240009383F300930190006316771A97200000C0
:10025000938040DB938000FE83D200029303F00F73
:100260009301A0006398721897200000938080D9B2
:100270009380B0FF83D27000B7030100938303F033
:100280009301B000639872169301C000130200003E
:1002900097200000938020D703D720001303070086
:1002A000B7130000938303FF631673141302120045
:1002B00093022000E31E52FC9301D00013020000C1
:1002C00097200000938040D403D720001300000043
:1002D00013030700B7F300009383F300631C73104C
:1002E0001302120093022000E31C52FC9301E00071
:1002F00013020000972000009380C0D003D7200095
:10030000130000001300000013030700B7030100EF
:10031000938303F06310730E130212009302200004
:10032000E31A52FC9301F000130200009720000032
:10033000938060CD03D72000B7130000938303FFA1
:10034000631A770A1302120093022000E31052FE90
:100350009301000113020000972000009380C0CA9F
:100360001300000003D72000B7F300009383F300CD
:10037000631277081302120093022000E31E52FC5E
:10038000930110011302000097200000938080C7A2
:10039000130000001300000003D72000B703010082
:1003A000938303F063187704130212009302200072
:1003B000E31C52FC972200009382C2C403D10200C6
:1003C00013012000930320009301200163147102A4
:1003D00097220000938202C303D1020013000000A1
:1003E0001301200093032000930130016314710076
:1003F000631030020F00F00F638001009391110031
:1004000093E111009308D0051385010073000000EB
:100410000F00F00F930110009308D00513050000A2
:1004200073000000731000C0000000000000000016
:0C043000000000000000000000000000C0
:1010000000000000000000000000000000000000E0
:1010100000000000000000000000000000000000D0
:1010200000000000000000000000000000000000C0
:1010300000000000000000000000000000000000B0
:081040000000000000000000A8
:10200000FF0000FFF00F0FF00000000000000000D4
:040000058000000077
:00000001FF
